:0200000480007A
:100000006F004005732F2034930F8000630AFF03B5
:10001000930F90006306FF03930FB0006302FF038A
:10002000170F0000130F0F2063040F0067000F006D
:10003000732F203463540F006F00400093E19153FD
:10004000171F000023203FFC171F0000232E0FFA6C
:100050006FF01FFF930000001301000093010000E8
:10006000130200009302000013030000930300003A
:100070001304000093040000130500009305000022
:10008000130600009306000013070000930700000A
:1000900013080000930800001309000093090000F2
:1000A000130A0000930A0000130B0000930B0000DA
:1000B000130C0000930C0000130D0000930D0000C2
:1000C000130E0000930E0000130F0000930F0000AA
:1000D000732540F16310050097020000938202012E
:1000E000739052307350447497020000938202015F
:1000F00073905230735000189702000093824202AE
:10010000739052309B021000939252039382F2FF3D
:100110007390023B9302F0017390023A73504030A7
:100120009702000093824201739052307350203046
:100130007350303093010000970200009382C2ECAC
:1001400073905230130510001315F501635C050020
:100150000F00F00F930110009308D0051305000065
:100160007300000093020000638A02007390521033
:10017000B7B200009B82921073902230735000300F
:10018000372500001B05058073200530970200000D
:100190009382420173901234732540F17300203032
:1001A0009301200013038000B72200009B8202808D
:1001B00073B00230F3230030B3F2720063840200A4
:1001C0001303B000B72200009B82028073B002309C
:1001D0009702000093820201739012347300203062
:1001E00093011000730000006F0080006310300264
:1001F0000F00F00F638001009391110093E1110053
:100200009308D00513850100730000000F00F00F64
:10021000930110009308D00513050000730000003F
:10022000F3222034F323503093F32300638403003C
:1002300093F2F20FE39E62FA970300009383C3FAEE
:10024000F3221034E39672FA6FF05FFC731000C073
:10025000000000000000000000000000000000009E
:10026000000000000000000000000000000000008E
:10027000000000000000000000000000000000007E
:1010000000000000000000000000000000000000E0
:1010100000000000000000000000000000000000D0
:1010200000000000000000000000000000000000C0
:1010300000000000000000000000000000000000B0
:081040000000000000000000A8
:040000058000000077
:00000001FF
